:100000000C946E040C94A6040C94A6040C94A60400
:100010000C94A6040C94A6040C94A6040C94A604B8
:100020000C94A6040C94A6040C94DF230C94B12425
:100030000C940D1F0C94A6040C94A6040C94A60416
:100040000C94A6040C94A6040C94A6040C94A60488
:100050000C94A6040C94951F0C94A6040C94A6046E
:100060000C94A6040C94A6040C94A6040C94A60468
:100070000C94A6040C94A6040C94A6040C94A60458
:100080000C94A6040C94A6040C94A6040C94A60448
:100090000C94A6040C94A6040C94A6040C94A60438
:1000A0000C94A6040C94A6040C94A6041A071A0730
:1000B00046074607BB08BB08BB08BB08AE07470896
:1000C000580858081E2545253D2645253D269125DD
:1000D000B4253D260B261A26556E6B6E6F776E0083
:1000E00041646A7573740044656661756C74003AA6
:1000F0000029001E001F002000210022003B002BD1
:100100000014001A000800150017003C00E100046C
:10011000001600070009000A003D00E0001D001B5A
:10012000000600190005000151E300E2002A002842
:10013000002C002D00C35C105000000000000000E7
:1001400000005CD35C0000C55CC65CC45C000000C1
:100150000000000000C95CC75CC85C000000000033
:10016000000000CB5C0000CA5C0000000001000041
:10017000000000000000000000000000010101017B
:100180000101010101020202020202020202030352
:100190000303030303030404040404040405050522
:1001A00005050606060606070707070708080808E4
:1001B000090909090A0A0A0B0B0B0C0C0C0D0D0D91
:1001C0000E0E0E0F0F0F1010111111121213131427
:1001D00014151516161717181819191A1A1B1B1C9F
:1001E0001D1D1E1E1F2020212222232424252626F9
:1001F000272829292A2B2C2D2D2E2F30313232332E
:100200003435363738393A3B3C3D3E3F4041424336
:100210004445464748494A4C4D4E4F50515354551A
:100220005658595A5B5D5E5F616264656668696BCA
:100230006C6D6F7072737577787A7B7D7E80828348
:100240008587888A8C8E8F91939596989A9C9EA08C
:10025000A2A3A5A7A9ABADAFB1B3B5B7BABCBEC099
:10026000C2C4C6C9CBCDCFD1D4D6D8DBDDDFE2E462
:10027000E7E9EBEEF0F3F5F8FAFDFF00AE00AF00B2
:10028000DA0281FFD9F1DB20A4A62EAF00A0C000C6
:10029000A1C800AED580A81FD300408D1420000750
:1002A000087F0807003E5B4F5B3E003E6B4F6B3E96
:1002B000001C3E7C3E1C00183C7E3C18001C577DF8
:1002C000571C001C5E7F5E1C0000183C180000FFDD
:1002D000E7C3E7FF00001824180000FFE7DBE7FF93
:1002E0000030483A060E00262979292600407F056D
:1002F000050700407F05253F005A3CE73C5A007F38
:100300003E1C1C0800081C1C3E7F0014227F221487
:10031000005F5F005F5F0006097F017F0000668964
:10032000956A0060606060600094A2FFA29400087B
:10033000047E04080010207E20100008082A1C08F3
:1003400000081C2A0808001E10101010000C1E0CBB
:100350001E0C0030383E383000060E3E0E060000FF
:10036000000000000000005F000000000700070020
:1003700000147F147F1400242A7F2A1200231308FC
:100380006462003649562050000008070300000050
:100390001C224100000041221C00002A1C7F1C2A54
:1003A0000008083E080800008070300000080808B7
:1003B0000808000000606000002010080402003EF1
:1003C0005149453E0000427F40000072494949467C
:1003D000002141494D33001814127F100027454574
:1003E0004539003C4A49493100412111090700368D
:1003F0004949493600464949291E000000140000B9
:1004000000004034000000000814224100141414BD
:100410001414000041221408000201590906003E8C
:10042000415D594E007C1211127C007F49494936CA
:10043000003E41414122007F4141413E007F494908
:100440004941007F09090901003E41415173007F84
:100450000808087F0000417F4100002040413F0123
:10046000007F08142241007F40404040007F021C72
:10047000027F007F0408107F003E4141413E007F23
:1004800009090906003E4151215E007F09192946EC
:100490000026494949320003017F0103003F4040E3
:1004A000403F001F2040201F003F4038403F006376
:1004B00014081463000304780403006159494D4390
:1004C00000007F414141000204081020000041412A
:1004D000417F00040201020400404040404000000F
:1004E00003070800002054547840007F2844443813
:1004F00000384444442800384444287F0038545489
:1005000054180000087E09020018A4A49C78007FFB
:10051000080404780000447D4000002040403D0075
:10052000007F102844000000417F4000007C0478D8
:100530000478007C0804047800384444443800FC03
:10054000182424180018242418FC007C080404082B
:100550000048545454240004043F4424003C4040C8
:10056000207C001C2040201C003C4030403C0044CB
:1005700028102844004C9090907C004464544C44D3
:1005800000000836410000000077000000004136FE
:100590000800000201020402003C2623263C000061
:1005A0000000000000404040F0F8F8FF38FFF8F885
:1005B0003FF8F8FF38FFF8F8F04040400000000036
:1005C000000080C0C0C0800000C0C080000000806B
:1005D000C0C000C0C0000080C0C00000000000C05B
:1005E000C0C0C0C000C0C00000000000000000008B
:1005F00000000000000000000000000000000000FB
:1006000000000000000000000000000000000000EA
:100610000000000000000000000000000000C0F02A
:10062000F8FC3E1E06010000007F4141417F007F33
:100630004141417F000080C0E07E5B4F5BFEC00017
:1006400000C000DCD7DEDEDED7DC00C0000000002A
:10065000000000000000000000000000000000009A
:100660000000000000494949FFFFFFFFE0DFBFBF76
:1006700000BFBFDFE0FFFFFFFF4949490000000066
:10068000001F3F6060E0BF1F007F7F071E381E070E
:100690007F7F007F7F0E1F3B716000000000007FA6
:1006A0007F0C0C0C007E7E007F7E0303007F7E03A8
:1006B000037E7E03037F7E000F3E703C063C703E4F
:1006C0000F00327B49493F7E007F7E0303001E3FBF
:1006D00069696F2600000000000000000000030FA1
:1006E0001F3F3C7870600000007F4141417F007FE8
:1006F0004141417F00307B7F7830202030787F3B44
:100700000003000F7F0F0F0F7F0F0003000000009A
:1007100000000000000000000000000000000000D9
:100720000000000000010101070F0F7F0F7F0F0F76
:100730007E0F0F7F0F7F0F0F0701010100000000E8
:1007400000000000000001010000000000000000A7
:100750000000000000000000000000000000000099
:100760000000000000000000000000000000000089
:100770000000000000000000000000000000000079
:100780000000000000000000000000000000000069
:100790000000000000000000000000000000000059
:1007A0000000000000000000000000000000000049
:1007B0000000000000000000000000000000000039
:1007C0000000000000000000000000000000000029
:1007D0000000000000000000000000000000001CFD
:1007E000034D006500630068004C006C0061006D03
:1007F0000061002000470033003500000010036B4B
:1008000000610079006C0079006E00620000000455
:1008100003090409023B00020100A0FA09040000D8
:100820000103010100092111010001224000070517
:1008300081030800010904010001030000000921EF
:1008400011010001223B0007058203200001120173
:10085000000200000008EBCE35000200010200019A
:1008600005010906A1018506050719E029E715001C
:1008700025019508750181020507190029EF15006A
:10088000250195F0750181020508190129059505D5
:1008900075019102950175039101C005010906A139
:1008A00001050719E029E715002501950875018163
:1008B000029501750881010507190029FF15002619
:1008C000FF009506750881000508190129059505A1
:1008D00075019102950175039101C00011241FBE9D
:1008E000CFEFDAE0DEBFCDBF04B603FE18C08091C3
:1008F0007E0490917F04A0918004B09181048730A0
:10090000904BA740B04B59F410927E0410927F0494
:100910001092800410928104E0E0F8E3099511E060
:10092000A0E0B1E0EEEEFDE402C005900D92A4332C
:10093000B107D9F724E0A4E3B1E001C01D92AE37BE
:10094000B207E1F70E945B140C94F5260C940000AA
:10095000882341F0813019F480EE90E0089588ED0D
:1009600090E0089587EE90E00895609151017091B4
:10097000520180915301909154010E948F050E9471
:10098000A80460E00E94F91880E0089581E00895CD
:1009900081E008950C94C80408950C94CC041F932E
:1009A000CF93DF9300D000D01F92CDB7DEB749833D
:1009B0005A836B833091370189819A81311114C038
:1009C000662359F0222349F00E94EC0A182F682F61
:1009D00089819A810E94950A03C00E94C00A182F3B
:1009E00069817A81812F04C00E94EC0A69817A8131
:1009F0000F900F900F900F900F90DF91CF911F915C
:100A00000C94F311FC01262F408151816281738186
:100A100084810C94CF0481E00895CF93DF93EC019F
:100A200060E00E940205BE01DF91CF910C94CD04DD
:100A30000C941F130C941B1308950E943F090E94ED
:100A40001C052FEF84E39CE0215080409040E1F7AB
:100A500000C000000C94BB1F0F931F93CF93DF9334
:100A60008C0161E00E940205EC01B8010E94CA04F9
:100A7000882309F444C0B801CE010E94581C882381
:100A8000F1F1B801CE010E946C1A8823C1F1B801BE
:100A9000CE010E94B41B882391F1B801CE010E94BF
:100AA000DD16882361F1F8018281882309F1CB35B5
:100AB0008DE5D807C1F050F4C115FCE5DF0781F0E2
:100AC000CF3DDC45A9F40E941D1019C0CC35EDE5E1
:100AD000DE0761F0CD35DD4559F40E94660F08C090
:100AE0000E941D050CC00E946F0F02C00E94720F71
:100AF000C801DF91CF911F910F910C94C60480E043
:100B0000DF91CF911F910F9108950E94F01E0E94D6
:100B1000F0050C94221A0E94F3050C94F61ECF9255
:100B2000DF92EF92FF926C01EE24FF24C114D104F6
:100B3000E104F10421F0C701B60120E101C020E089
:100B4000C72ED82EE92EFF24C114D104E104F104EC
:100B500019F0285FC701B6016B017C0154E0F694DF
:100B6000E794D794C7945A95D1F7C114D104E104FE
:100B7000F10419F02C5FC701B6016B017C0142E062
:100B8000F694E794D794C7944A95D1F7C114D10449
:100B9000E104F10419F02E5FC701B601DC01CB01BD
:100BA000B695A79597958795892B8A2B8B2B09F05E
:100BB0002F5F822FFF90EF90DF90CF9008950895E0
:100BC0000C94DF0581E008950C94E2050895CF931D
:100BD000C82F0E94E0058C2F0E94E405CF91089554
:100BE00080E00C94E7050E94C31D0C94E7050E9469
:100BF000C31D90913601891721F0809336010C9422
:100C0000E7050895CF93DF93CDB7DEB72B970FB6E7
:100C1000F894DEBF0FBECDBF4F83588769877A87B0
:100C20008B8761110E94B20E9E012F5F3F4F86E0BD
:100C3000F90111928A95E9F785E0FE013796D9010D
:100C400001900D928A95E1F789819A814C815D81AD
:100C5000452B31F09F3F31F491E08F3F19F403C0F1
:100C600091E001C090E090FF09C049815A816B81F9
:100C70007C818D819E810E94D30D05C0C9010E9497
:100C80000B058111F2CF2B960FB6F894DEBF0FBE85
:100C9000CDBFDF91CF910895FC01808191810E94A9
:100CA0002E0B0895CF93882371F1C82F8CEF8C0FF2
:100CB000813AD0F46C2F80910201909103010E943F
:100CC0002B1E882349F06C2F809102019091030123
:100CD0000E94B61E0E94D40E6C2F8091020190914A
:100CE00003010E94AB1E0CC080E28C0F883058F4C8
:100CF000C77081E001C0880FCA95EAF70E94950E7F
:100D0000CF910C94D40ECF910895882349F1682F88
:100D10008CEF860F813A38F48091020190910301A3
:100D20000E94B61E0CC080E2860F883050F46770B7
:100D300081E001C0880F6A95EAF70E949B0E0C942F
:100D4000D40E8BE5860F833020F480E090E00C9485
:100D5000E91D685A673120F480E090E00C94FF1D93
:100D600008951F93CF93DF93182FEB010E94520633
:100D7000209741F08FE99FE00197F1F700C0000054
:100D80002197F6CF812FDF91CF911F910C9485068B
:100D9000893319F060E070E002C060E570E00C9407
:100DA000B106882321F00E94950E0C94D40E08956C
:100DB000882321F00E949B0E0C94D40E0895CF92AC
:100DC000DF92EF92FF920F931F93CF93DF937C01FB
:100DD000D62FC72FFC011281058102950F700E944A
:100DE0008B0E8823B9F01123A9F08C2F807F8034DB
:100DF00021F080E28D0F883068F08091450282FDFD
:100E000009C082E00E94340F0E948B0E91E0D82E20
:100E1000D92601C0D12CCC2EC2948FE0C8228C2DB3
:100E200090E08C30910508F0A6C1FC01EA5AFF4F12
:100E30000C9491268C2F807FCF70882311F0C2955F
:100E4000C07F112399F0CC2309F481C180E28D0F7A
:100E5000883010F0D11104C08C2F0E94950E03C071
:100E60008C2F0E94A50E0E94D40E71C18D2F0E945E
:100E70008506CC2309F47FC180E28D0F883038F1DC
:100E8000DD2329F18C2F0E94AB0E24C08C2F807F94
:100E9000CF70803211F0C295C07FDD2319F0D130C0
:100EA000A1F13DC08091450282FF17C0112349F096
:100EB000CC2329F08C2F0E94950E0E94D40E80E046
:100EC00047C180E00E948506CC2309F454C18C2FD1
:100ED0000E949B0E0E94D40E4EC1112371F000237C
:100EE00041F0013031F40E94B50E8C2B0E94BD0EF2
:100EF00042C10E94B50E8C2B1DC0002319F0013099
:100F000009F439C10E94CA0E25C0112321F0063010
:100F100008F031C10EC0053008F02DC11BC01123EF
:100F200061F0002331F0F701858180FF10C18F70DF
:100F300085838C2F0E94D1061EC1002359F0D9331E
:100F400009F016C1FFEF07EE13E0F150004010402A
:100F5000E1F70CC18C2F0E94D8060DC18C2F837035
:100F600009F047C011110BC12D2F2295269527702E
:100F7000220F220F6D2F6F70862F90E0A0E0B0E05F
:100F8000022E04C0880F991FAA1FBB1F0A94D2F714
:100F9000D4FF10C04FE050E060E070E004C0440FA8
:100FA000551F661F771F2A95D2F74095509560957B
:100FB000709503C040E050E0BA01C695C695C37075
:100FC0008A019B01082B192B2A2B3B2BC901B80145
:100FD000C23049F058F4C13019F00E94AB09CFC0BB
:100FE0000E949909CCC00E94BD09C9C00E949709FE
:100FF000C6C0112319F08C2F817001C086958823FB
:1010000009F4BDC02D2F229526952770220F220F9F
:101010006D2F6F70862F90E0A0E0B0E0022E04C02C
:10102000880F991FAA1FBB1F0A94D2F7D4FF10C0C4
:101030004FE050E060E070E004C0440F551F661FB1
:10104000771F2A95D2F7409550956095709503C00B
:1010500040E050E0BA01C695C695C3708A019B0175
:10106000082B192B2A2B3B2BC901B801C23049F0A0
:1010700058F4C13019F00E94700A81C00E945E0AC3
:101080007EC00E94820A7BC00E94D10978C0CF70C6
:10109000112339F08C2F0E94F7098D2F0E94D10661
:1010A0006EC08D2F0E94D8068C2F0E94180A67C030
:1010B000D23F21F128F4D03F41F0D13FC1F043C0ED
:1010C000D33F19F1D43F79F03EC0112341F00530F0
:1010D00008F051C08C2F8F710E943D0A4CC0063021
:1010E00008F049C0F7CF8091450282FF18C0112354
:1010F00039F08C2F8F710E94F7093DC01123C9F37D
:101100008C2F8F710E94180A36C0112329F08C2F62
:101110008F710E94E2092FC00E94DD092CC01123AB
:1011200049F0CF718C2F0E94F70963E08C2F0E9449
:10113000190F21C081E00E94340F0230E0F082E0FC
:101140000E94340F18C0112331F0002391F28D2F2B
:101150000E94520610C0002399F2D93349F41FEFC0
:1011600027EE33E0115020403040E1F700C000008E
:101170008D2F0E94850688EF8C0D843020F40E940C
:10118000C31D0E94E705DD20C9F00E94870E80FD87
:1011900015C0F70112820E94810E0E94F709C70153
:1011A0000E94FF080E94810EDF91CF911F910F9145
:1011B000FF90EF90DF90CF900C94180ADF91CF91C1
:1011C0001F910F91FF90EF90DF90CF9008950F93B4
:1011D0001F93CF93DF93EC01688179818A810E940C
:1011E000390B8C010E94940A0E948509B801CE0136
:1011F0000E94DF06DF91CF911F910F910895CF9349
:10120000DF93EC01988189812B813C81232B31F084
:101210008F3F31F481E09F3F19F403C081E001C0AA
:1012200080E080FD1DC0CE010E942C05811110C000
:101230000E948B0E8823A1F08A81882389F08091F7
:10124000450282FD0DC082E0DF91CF910C94340FF6
:10125000CE010E94E708CE01DF91CF910C940D05DD
:10126000DF91CF9108950E94B20E0C94D40E80911C
:101270000201909103010E94C11E0C9433090E9447
:10128000A20E0C94370992959F70963079F010F465
:10129000925001C09A50923068F4803F69F018F47F
:1012A000883E40F409C0843F29F406C0883E20F0FF
:1012B000813F11F080E0089581E00895FC01808174
:1012C00091810E942E0B0E9443090895CF93DF93D2
:1012D00000D000D01F92CDB7DEB70F900F900F90C7
:1012E0000F900F90DF91CF910895CF93DF9300D0AF
:1012F00000D000D0CDB7DEB726960FB6F894DEBF8B
:101300000FBECDBFDF91CF910895089508950C943D
:1013100086090C9487090E9489096093550170938E
:10132000560180935701909358010C9433090C9403
:101330008B090F931F930091550110915601209135
:10134000570130915801602B712B822B932B1F91E9
:101350000F910C948B090F931F93009155011091DD
:101360005601209157013091580160237123822347
:1013700093231F910F910C948B090F931F9300914E
:101380005501109156012091570130915801602765
:101390007127822793271F910F910C948B090C942E
:1013A00086090E94CF096093510170935201809386
:1013B0005301909354010C94330960E070E0CB0129
:1013C0000C94D1090F931F9341E050E060E070E06E
:1013D0008A019B0104C0000F111F221F331F8A9531
:1013E000D2F7C901B8011F910F910C94D1090F9345
:1013F0001F9341E050E060E070E004C0440F551FCF
:10140000661F771F8A95D2F7809151019091520102
:10141000A0915301B09154018A019B01082B192B13
:101420002A2B3B2BC901B8011F910F910C94D109B4
:101430000F931F9341E050E060E070E004C0440F60
:10144000551F661F771F8A95D2F740955095609576
:1014500070958091510190915201A0915301B091EA
:1014600054018A019B01082319232A233B23C90124
:10147000B8011F910F910C94D1090F931F9341E074
:1014800050E060E070E004C0440F551F661F771FF6
:101490008A95D2F78091510190915201A091530108
:1014A000B09154018A019B01082719272A273B275D
:1014B000C901B8011F910F910C94D1090F931F938B
:1014C000009151011091520120915301309154012A
:1014D000602B712B822B932B1F910F910C94D109B0
:1014E0000F931F93009151011091520120915301CC
:1014F0003091540160237123822393231F910F9114
:101500000C94D1090F931F93009151011091520136
:10151000209153013091540160277127822793272E
:101520001F910F910C94D109089527E0929F800D8F
:101530001124E82FE695E695E695877051E001C005
:10154000550F8A95EAF785E0E89FF0011124E85CE1
:10155000FE4F20E030E070E04081CB01022E02C05F
:10156000969587950A94E2F7817081958427852363
:10157000842781932F5F3F4F2530310569F7089508
:1015800027E0929F800D1124682F669566956695D9
:10159000982F977085E0689FB001112440E050E0DB
:1015A00080E0FB01E40FF51FE85CFE4F208130E096
:1015B000092E02C0369527950A94E2F72170332749
:1015C000042E01C0220F0A94EAF7822B4F5F5F4F6F
:1015D0004530510531F70895BF92CF92DF92EF92D7
:1015E000FF920F931F93CF93DF938C01C090510113
:1015F000D0905201E0905301F09054018091550138
:1016000090915601A0915701B0915801C82AD92A4A
:10161000EA2AFB2ACFE1D0E0D701C6010C2E04C094
:10162000B695A795979587950A94D2F780FD04C043
:10163000219790F7B12C07C0BC2EB8018C2F0E94C7
:1016400006120197A9F38B2DDF91CF911F910F9176
:10165000FF90EF90DF90CF90BF900895CF93DF93EE
:10166000EC010E94EC0ABE010E940612DF91CF91AC
:1016700008951F93CF93DF93EB0190913701992346
:1016800021F0CB010E942E0B13C0882349F0CB011F
:101690000E94EC0A182F682FCE010E94950A04C000
:1016A000CB010E94C00A182FBE01812F0E94061292
:1016B000DF91CF911F9108951F93CF93DF93C09136
:1016C000590116E080915A01C81799F0D0E01C9F8B
:1016D000F0011D9FF00D1124E55AFE4F408151810C
:1016E00062817381848195810E9475092196C770FA
:1016F000E9CFDF91CF911F91089540918B015091D7
:101700008C0160918D0170918E0180918F0190917B
:1017100090010C947509EF92FF920F931F93CF9352
:10172000DF938091900182958F7009F065C0809160
:101730008D01882309F460C080915901F0905A010D
:1017400010918B0100918C0160918E0170918F013D
:1017500091E01F3F09F090E0C0910001D09101019C
:10176000292F96E0E92E8F1509F446C06115710501
:1017700021F00F3F21F030E003C031E001C0322FF3
:1017800090E030FD36C0E89EF001E99EF00D112496
:10179000DF01A55ABE4F11963C911197301329C015
:1017A0003C91311326C012963C911297311121C001
:1017B00013964D915C911497461B570B4C175D0780
:1017C000C0F4809190018F70806180939001E05A05
:1017D000FE4F80818F70806180838BE891E00E9452
:1017E000FF08DF91CF911F910F91FF90EF900C9424
:1017F0005C0B01968770B7CFDF91CF911F910F914E
:10180000FF90EF9008959F92AF92BF92CF92DF9298
:10181000EF92FF920F931F93CF93DF93CDB7DEB775
:1018200061970FB6F894DEBF0FBECDBF8C0185E087
:10183000F801DE011D9601900D928A95E1F7D8011D
:101840001296EC9090918B01E0918C0120918E0189
:1018500030918F012115310531F0EF3F31F481E0F6
:101860009F3F19F403C081E001C080E0B82FB17040
:101870009B2E80FD47C1D8014C9111965C91119728
:101880001396AD90BC9014978BE8C82E81E0D82EAB
:10189000F0908D01B501621B730B20910001309116
:1018A0000101FF2009F4D9C08091900162177307EC
:1018B00008F095C0282F207F09F052C05E1313C096
:1018C000491311C0FE2CE1100EC08F70806180930F
:1018D00090010E947D0BC6010E94FF08809190013B
:1018E000F80185834DC1AB2831F05F3F31F481E0D1
:1018F0004F3F19F403C081E001C080E080FD03C0C8
:1019000081E08E2502C080E090E0F82FF170FF2E7C
:1019100080FF1CC08091590120915A0136E0821746
:1019200009F40BC190E0389FF001399FF00D1124AC
:10193000E55AFE4F6181561306C06081461303C00D
:101940006281E61203C001968770E9CFFE2CEE207B
:1019500009F416C18091900181608093900154C078
:101960005E1306C0491304C0E11002C0F80199C01B
:10197000C8010E945E09882361F1EE2051F1209197
:101980009001822F82958F7090E0029774F0809181
:101990008B0190918C0198878F831986BB86AA86CC
:1019A0002C87CE0107960E94FF0886E0F801ABE87D
:1019B000B1E001900D928A95E1F70E948B0B0E9495
:1019C0007D0B0AC05E1711F1C8010E945E098111EA
:1019D0002CC0C8010E94FF08FF24F394D1C0282F17
:1019E000207F81F77A2DB98AA88A6E2D89890E9475
:1019F00066098BE891E00E94FF0886E0D6011D92FF
:101A00008A95E9F70E947D0BF12CBAC04913DCCF0F
:101A1000E110DACFF8018583C8010E94FF0886E053
:101A2000D6011D928A95E9F7ABC0EE2091F2209184
:101A30009001822F82958F7090E002970CF4B5CFC1
:101A400080918B0190918C019A8389831B82BD8246
:101A5000AC822E83CE010196A6CF6217730708F0E1
:101A600044C0FE2CEE2009F4B4CF5E1330C04913FD
:101A70002EC02091900120FD21C0822F82958F7071
:101A8000482F50E041155105C9F0F80125834F302A
:101A9000510541F08F5F982F9295907F822F8F7024
:101AA000892B8583C8010E94FF0886E0F801ABE816
:101AB000B1E001900D928A95E1F73CC086E0F80113
:101AC000ABE8B1E001900D928A95E1F759C0C801E9
:101AD0000E945E09811169CF80919001816080939D
:101AE0009001C8010E94FF084BC07A2DB98AA88ACC
:101AF0006E2D89890E94660986E0D6011D928A951D
:101B0000E9F718C0EE2009F464CFC8010E945E090D
:101B1000F82E882309F45DCF86E0F801ABE8B1E048
:101B200001900D928A95E1F78BE891E00E944C06B6
:101B30000E948B0B0E947D0B23C04D875E878D8595
:101B40009E850E942E0B292F22952F70223028F47B
:101B50009F7039F0811105C00BC0243028F49F70AC
:101B600049F4805E883020F0C8010E94FF089F2C55
:101B7000F92C06C0D80115969C91907F91F7F8CF6B
:101B80008F2D61960FB6F894DEBF0FBECDBFDF91EB
:101B9000CF911F910F91FF90EF90DF90CF90BF906A
:101BA000AF909F9008951F93CF93DF93CDB7DEB78B
:101BB0002C970FB6F894DEBF0FBECDBF4F8358876A
:101BC00069877A878B879C87CE0107960E94030CD2
:101BD0008823D1F09F8188852A853B85232B31F08E
:101BE0008F3F31F481E09F3F19F403C081E001C0D1
:101BF00080E080FD47C04F81588569857A858B8557
:101C00009C850E9475093EC086E0FE013796DE0184
:101C1000119601900D928A95E1F7FF81E8856A851A
:101C20007B856115710531F0EF3F31F481E0FF3FB5
:101C300019F403C081E001C080E080FD23C0209141
:101C40005A0130E0C90101968770992740915901E6
:101C500050E084179507F1F1F983EA837D836C8363
:101C600096E0929FD001939FB00D1124A55ABE4FCC
:101C7000FE01319601900D929A95E1F780935A01F9
:101C80000E945C0B16E08091590190915A018917CE
:101C900071F1189FC0011124855A9E4F0E94030CB8
:101CA000882329F1E09159011E9FF0011124E55A82
:101CB000FE4F4081518162817381848195810E94B0
:101CC00075098091590190E001968770992780935A
:101CD0005901D9CF0E943F0910925A01109259011F
:101CE000EBE8F1E086E0DF011D928A95E9F72C969A
:101CF0000FB6F894DEBF0FBECDBFDF91CF911F911D
:101D000008958091B1018595859585950895809177
:101D1000B101877008959091B101977081E009F445
:101D200080E008958091D40108959091D401892B89
:101D30008093D401089580959091D4018923809354
:101D4000D40108951092D40108959091D301892B64
:101D50008093D301089580959091D3018923809336
:101D6000D30108951092D30108958091B20108958E
:101D700008950C94B80E0C94B90E9091450292FD02
:101D800008C09091B201981721F08093B2010C9491
:101D9000BB0E08958091B201882329F01092B20100
:101DA00080E00C94BB0E0895CF93DF93E091020185
:101DB000F09103018091D4018083E0910201F091C0
:101DC000030190818091D301892B80838091B2019E
:101DD000882381F0E0910201F09103019081892B29
:101DE000808380910201909103010E94151E811150
:101DF0000E94CA0EC0910201D091030140E250E05E
:101E000061E971E0CE010E94A026892B69F080E291
:101E1000FE01A1E9B1E001900D928A95E1F7CE01B2
:101E2000DF91CF910C94CF1DDF91CF9108950C9449
:101E3000B80E9091450292FD10C098E0899F9001E4
:101E40001124262B2093B1010E94F7098091B10142
:101E50008595859585950C94170F0C94F70910922C
:101E6000B10180E00C94170F2091B101809582237D
:101E70008093B101982F977099F430E0482F082E85
:101E8000000C550B2417350759F09091450292FD2F
:101E900007C08595859585950E94180A0C942F0F8B
:101EA00008959091450292FB222720F9281769F0A6
:101EB00080FB92F9909345028091440290914502F3
:101EC0000E94990F82E00C94340F0895809145028E
:101ED00082FB882780F991E089270C94510F81E0DB
:101EE0000C94510F80E00C94510F80E090E00E9420
:101EF000BB2621E0893E9E4F09F020E0822F089505
:101F000082E090E00C94AD2683E090E00C94AD2646
:101F1000CF9384E090E00E94AD26C82F82E290E04B
:101F20000E94AD262C2F30E0A901582BCA01CF9179
:101F30000895CF93C92F682F84E090E00E94C126B6
:101F40006C2F82E290E0CF910C94C126AB01BC01D2
:101F50008FE090E00C94D326AB01BC0183E190E0CC
:101F60000C94D32660E070E0CB010C94AC0F60E0E1
:101F700070E0CB010E94A60F0C94B20F69EE7EEFC9
:101F800080E090E00E94DF2660E082E090E00E9426
:101F9000C12660E083E090E00E94C12610925501C6
:101FA00010925601109257011092580160E084E09F
:101FB00090E00E94C12660E082E290E00E94C1268B
:101FC00060E085E090E00E94C12660E086E090E05D
:101FD0000E94C1266FEF87E090E00E94C12640E09A
:101FE00050E0BA0188E090E00E94D32660E08DE0E6
:101FF00090E00E94C12640E050E0BA0188E190E004
:102000000E94D32660E087E190E00E94C12640E074
:1020100050E0BA018CE190E00E94D32660E070E0CD
:1020200080E290E00E94DF2640E050E0BA0188E1C3
:1020300090E00E94D3260C94B70F0C94BE0F682F2B
:102040008EE090E00C94C1260E947A1F6093DE011E
:102050007093DF018093E0019093E1016093DA01D6
:102060007093DB018093DC019093DD01089585B7C7
:10207000806885BF85B7806885BF089581E0089531
:102080000C943E1008950C9442100C9442100C9441
:1020900045100C9442100C9449100C9442100E946C
:1020A000371082EE92E10E94B91D0E944D100C94EF
:1020B0004B100E9443100C9442100E94E5120C94A5
:1020C000E6050E94651F0E94BC130E945D1080E01F
:1020D0000E94C0170E94A616E4E4F2E080818068A6
:1020E000808380914402909145020E94990F0C9444
:1020F00047108F929F92AF92BF92CF92DF92EF9252
:10210000FF920F931F93CF93DF93CDB7DEB72A973C
:102110000FB6F894DEBF0FBECDBF0E94D113982E2C
:1021200081110E94241085EDA82E81E0B82E00E0D8
:1021300010E0802E802F0E940913D82EF501C19047
:102140005F01C826B1F40F5F1F4F0530110589F7F5
:102150008FEF89838A831B820E946E1F8160782F94
:102160009D838C8349815A816B818D810E940206F7
:102170002FC08091E20181FD0E940F13E12CFF240A
:10218000F3948C2D8F21F1F00E944010882399F058
:10219000EE828F82DF2081E009F480E088870E9450
:1021A0006E1F8160782F9A8789874E815F8168854D
:1021B0008A850E940206F801EB52FE4F8081F826C4
:1021C000F08206C0E394FF0CF7E0EF12DACFBBCF4A
:1021D00081E0911001C080E02A960FB6F894DEBF2E
:1021E0000FBECDBFDF91CF911F910F91FF90EF9068
:1021F000DF90CF90BF90AF909F908F900895CF9336
:102200000E947910C82F0E943E1AC1110E94FE1828
:10221000CF910C94F705CF93DF930E940B12EC0142
:10222000811523E59207A0F5811532E5930708F0A3
:102230009EC0811540E29407C0F4811551E09507D6
:1022400008F0CDC0853A910550F48430910508F02E
:10225000C6C0019709F0C0C081E090E0C1C0805EB7
:102260009109089708F4BBC0B7C0C11581E5D8072C
:1022700008F077C0C11520E5D20708F051C0C1159C
:1022800030E4D30708F4A8C0DF70CE01906AA8C07C
:10229000811546E5940700F5811555E5950708F089
:1022A00081C0C11584E5D80708F076C0CE018370DF
:1022B000992721E030E002C0220F331F8A95E2F710
:1022C0009C2F9695969540E2949FE0011124C22B95
:1022D000D32BCE019A6884C081152AE5920780F439
:1022E000811539E5930708F066C0811548E5940724
:1022F00008F472C0D82FCC27CE01806F906A70C0CE
:1023000090568115904208F067C08D2F8F710E9402
:102310009F12DD27D0628F71AE01582BCA0160C0B9
:10232000CE0174E0969587957A95E1F7282F237072
:102330003C2F337081E090E002C0880F991F3A95DE
:10234000E2F79C68AC01522B9A019C2F9F709695E6
:10235000969550E2959FE0011124C9018C2B9D2B8D
:102360003FC0DC2FCC27CE01816F906A39C08370CB
:10237000992721E030E002C0220F331F8A95E2F74F
:102380009C2F9695969580E2989FE0011124C22B90
:10239000D32BCE019C6824C0DC2FCC27CE01846FC8
:1023A000906A1EC00E949F128F7190E0D82FCC2798
:1023B000CE01906215C08F700E949F1294E0D69556
:1023C000C7959A95E1F7CF70D0E0DC2FCC27D06984
:1023D0009E01282BC90104C080E090E001C0CE011D
:1023E000DF91CF91089523E2829FC0011124FC0167
:1023F00027E0729FE00DF11D1124E60FF11DEE0F95
:10240000FF1FE151FF4F8591949108950E94F311B0
:102410000E940B1108958238910569F1B0F481335F
:10242000910509F46DC048F48932910509F463C03F
:102430008A32910509F469C008958533910509F43C
:1024400055C089339105B9F00895833E910569F12E
:1024500038F4803E9105B1F0823E910509F108956E
:10246000863E9105A9F1873E9105B9F1843E91051B
:1024700009F064C023C02091440220FD4FC021FD1B
:102480004DC008958091440280FD44C08091450272
:1024900080FF44C08091440284FD42C083EE4DC061
:1024A0008091440282FF38C0F5CF8091440282FDC2
:1024B00033C08091450280FD31C0ECCF8091450250
:1024C00081FF32C08091440284FD2AC087EE35C06E
:1024D0008091440283FF26C0F5CF8091440283FDA2
:1024E00021C08091450281FD1FC0ECCF8091440244
:1024F00085FD1CC01DC08091440285FD19C016C019
:102500008091440286FD16C017C08091440286FD6A
:1025100013C010C089E311C082EE0FC080EE0DC061
:1025200080E00BC086EE09C084EE07C089E205C0DA
:1025300085E303C08AE201C081E390E008959091B1
:10254000440292FF0DC0282F2871283019F4877F8C
:10255000846006C0282F2471243011F48B7F88609A
:1025600093FF0DC0282F2871283119F4877E8461CC
:1025700006C0282F2471243111F48B7E88612091AC
:10258000450220FF0DC0382F3871383019F4877F8D
:10259000816006C0382F3171313011F48E7F886030
:1025A00021FF0DC0282F2871283119F4877E816101
:1025B00006C0282F2171213111F48E7E886194FD8F
:1025C000877E089580E0089508950E94750F811117
:1025D00002C00E941D100E94800F8093E2010E94A1
:1025E000880F90934502809344020E94E4120E9457
:1025F000840F682F70E080E090E00E94970960915E
:1026000051017091520180915301909154010C94A9
:10261000CF09E82FF0E0E55BFD4F80810895089534
:1026200080EA8A95F1F7089500C008950C9410137C
:1026300008950C9418130C9419130C9418130C94FB
:102640001D13F894E82FE295EF70F0E031A1282FE8
:102650002F7081E090E001C0880F2A95EAF7982F4B
:102660009095932391A392A1892B82A378940895A6
:102670000F931F93CF93DF93C4E2D1E089918F3FF3
:1026800011F00E94211381E0C932D807B9F7CDE1DA
:10269000D1E004E211E089918F3F11F00E942113F3
:1026A0000C171D07C1F7DF91CF911F910F9108956E
:1026B000CF92DF92EF92FF920F931F93CF93DF930E
:1026C0008C01C62FD0E0CE018C5D9E4F7C01FC01B9
:1026D00090819F3F09F447C0D62EF894E92FE295E8
:1026E000EF70F0E081A19F7021E030E001C0220F87
:1026F0009A95EAF7822B81A382A12095282322A311
:1027000078940E941413EDE1F1E044E251E031E0ED
:10271000C12C21912F3F89F0A22FA295AF70B0E07C
:1027200090968C9190E02F7002C0959587952A9590
:10273000E2F780FD02C0832F01C080E0C82A330F7A
:102740004E175F0731F7F70180818F3F11F00E942C
:10275000211361E0C11001C060E08D2D0E941613AD
:10276000C00FD11FC882DF91CF911F910F91FF90B1
:10277000EF90DF90CF9008950E94381385E0EBE44E
:10278000F2E0DF01982F1D929A95E9F7E6E4F2E076
:10279000DF011D928A95E9F785E00E9418140C94D8
:1027A0001805FF920F931F93CF93DF9300D000D0B3
:1027B0001F92CDB7DEB78E010F5F1F4F85E0F80186
:1027C00011928A95E9F7F12C6F2DC8010E945813D8
:1027D000F394F5E0FF12F8CF45E050E0B80186E44D
:1027E00092E00E94A026FF24F394009709F4F12CB4
:1027F000892B41F085E0F801A6E4B2E001900D924A
:102800008A95E1F72F2D45E06BE472E086E492E0D3
:102810000E9419140E941A058F2D0F900F900F908F
:102820000F900F90DF91CF911F910F91FF9008951E
:102830000895FF920F931F93CF93DF938C01F62E91
:10284000D72FC42F222349F081E08093E5010E9415
:102850006E1F9093E4018093E3018091E50188234A
:10286000C1F08091E3019091E4010E94861F0597D9
:1028700080F0EF2DFD2FD8014C2F50E0CD01801BB3
:10288000910B841795071CF48D918193F7CF1092CB
:10289000E501DF91CF911F910F91FF9008950E9464
:1028A00037210E9461100C9443210E9447210E940D
:1028B000FF100C9461210E940C1F0E941E210E9497
:1028C0004F100E944F140E9455140E945910FBCFC4
:1028D000EF92FF920F931F93CF93DF938B01682F9B
:1028E00011110AC0442329F0E82FF0E0E558FE4F0B
:1028F0006491762F862F75C0212F30E0E82FF0E00D
:10290000442321F0E558FE4FE491F0E046E0049FB7
:10291000C0011124CFEFD0E0BE010E947D264BEA1A
:102920004603C001479F900D1124800F911D800F19
:10293000911D982F990F890FAE01421B530B4E9F8B
:10294000D0014F9FB00D5E9FB00D11249B2F189F9B
:10295000A0011124452F55278E01041B150B0E9F36
:10296000A0010F9F500D1E9F500D11247E01E81AEB
:10297000F108E29E8001E39E100DF29E100D1124DD
:10298000212F3327C21BD30BCE9F9001CF9F300D39
:10299000DE9F300D112462307105A9F048F46115F5
:1029A000710569F061307105C9F48B2F752F0DC069
:1029B0006430710581F058F06630710579F47E2F2E
:1029C0008B2F932F0DC0832F7B2F9E2F09C08E2F0F
:1029D0007B2F952F05C08E2F732F02C07E2F852F42
:1029E000692FDF91CF911F910F91FF90EF90089584
:1029F00041E00E94681408950E94F8140895CF934E
:102A0000DF93762FE901682F842F0E94FC147983CD
:102A100068838A83DF91CF91089580915002982F27
:102A20009695913021F081708260809350020895D4
:102A300088E090E00C94B526CF92DF92EF92FF925F
:102A40006B017C010E940D15B701A60188E090E0A2
:102A5000FF90EF90DF90CF900C94D326E0E5F2E06A
:102A600083E0808311828FEF82838383148260816D
:102A70007181828193810C941C1590915402933042
:102A800018F49F5F90935402882351F06091500294
:102A90007091510280915202909153020C941C1536
:102AA000089581E00C943D1590915402992319F0FA
:102AB000915090935402882351F06091500270918C
:102AC000510280915202909153020C941C1508956A
:102AD00081E00C94541570E00C945417609105013A
:102AE0008091500280FF0AC08091040123E0829F00
:102AF000C00111248B5A9D4F0C946B1580910601D7
:102B000090910701891780F7E82FF0E09F01220FCD
:102B1000331FE20FF31FEB5AFD4F11821082128216
:102B20008F5FF0CFE0E5F2E080818E7F808360816F
:102B30007181828193810E941C152FEF80E792E0C2
:102B4000215080409040E1F700C000000C946E15C9
:102B50009091500290FF16C09091060120910701BC
:102B6000921770F4E92FF0E0DF01AA0FBB1FEA0F04
:102B7000FB1FEB5AFD4F8183608342839F5FF0CF41
:102B80000C946E150895EF92FF920F931F93CF93BD
:102B9000DF9300D01F92CDB7DEB79091500290FF27
:102BA0002CC0E22E142F062FF82EE92FE695F0E028
:102BB000E75DFE4F80818093E7019E7F923059F45C
:102BC0009E012F5F3F4F8F2D0E94FF144B81698123
:102BD0008A810E94A815F09251020093520210932C
:102BE0005302EE2051F06091500270915102809199
:102BF0005202909153020E941C150F900F900F905B
:102C0000DF91CF911F910F91FF90EF900895E0E534
:102C1000F2E09181282F4381628188E0890F0C9432
:102C2000C31581E00C940716E0E5F2E09181282FAE
:102C30004381628188EF890F0C94C31581E00C9465
:102C40001416E0E5F2E0628121E1620F08F46FEF13
:102C5000282F438181810C94C31581E00C942116A7
:102C6000E0E5F2E0628121E1621B08F460E0282FD8
:102C7000438181810C94C31581E00C943016E0E50A
:102C8000F2E0438121E1420F08F44FEF282F6281E7
:102C900081810C94C31581E00C943F16E0E5F2E0CD
:102CA000438121E1421B08F440E0282F62818181A9
:102CB0000C94C31581E00C944E1620E00C94C315BF
:102CC0008091500280FF18C0817082608093500212
:102CD000662351F06091500270915102809152022E
:102CE000909153020E941C15409153026091520230
:102CF000809151020C945D160895682F81E00C9428
:102D0000601681E00C947D16682F90915002969584
:102D10008FEF890F09F481E00C94601681E00C9428
:102D2000841661E00C946016E0E5F2E08081816039
:102D3000808386950C9491168091500280FD0C94AE
:102D400092150C94941660E00C9460168091E60144
:102D500081112CC00E94750F811104C00E941D10AA
:102D60000E942E150E941815609350027093510214
:102D700080935202909353026E7F61F40E942E154D
:102D80000E94181560935002709351028093520272
:102D9000909353020E940D158091500280FF03C052
:102DA00086950E94A31681E08093E601089588230A
:102DB00011F0FA0101C0FB0109941F93CF93DF9337
:102DC000FB01128111116BC0EC010E94920E827204
:102DD000CA3CFCE5DF0709F450C0C0F4C63CECE592
:102DE000DE07E1F148F4C43C9CE5D90759F178F5D8
:102DF000C33CDC4521F121C0C83C9CE5D90799F1D1
:102E0000B8F541E156E16EE176E125C0CE3CFCE546
:102E1000DF0709F441C050F4CC3CECE5DE0791F14A
:102E2000B0F54BE456E16AE576E115C0C73D8CE5A7
:102E3000D807A8F1CE35DD4591F111E030C00E94F0
:102E40009C162DC04EE856E161E876E104C041E8E9
:102E500056E16EE876E10E94D71621C04EE156E1B8
:102E600061E176E1F8CF4CE356E16DE276E1F3CF34
:102E70004DE256E16CE376E1EECF4AE556E16BE4D4
:102E800076E1E9CF48E655E161E575E1E4CF41E55A
:102E900055E168E675E1DFCF81E00E949116812F50
:102EA000DF91CF911F910895879A21B32F7731B386
:102EB00030684FB7F894FC01CB01880F991F680F59
:102EC000791F6E0F7F1FE617F70789F0819198E051
:102ED00031BB000000C087FF21BB880F000000C08D
:102EE00000C000C021BB00C09A9591F7ECCF4FBF46
:102EF0008FE594E00197F1F700C000000895EF928C
:102F0000FF920F931F93CF93DF93EC017B0164E655
:102F100070E088E70E94B01C8C01EC0EFD1ECE15FF
:102F2000DF0561F017FD0AC0FE01849164E670E0E0
:102F30000E94311D8C012196892B89F30E94B51DB9
:102F4000C801DF91CF911F910F91FF90EF900895ED
:102F500008950C94A817E7E6F2E080E092E0DF0124
:102F60009C011D9221503040E1F7F0936C04E093F6
:102F70006B048FEF9FEF90931502809314020895D6
:102F80000E94A9170E94A8178093100280FD02C01A
:102F900080E801C080E280930F020E94AA1C6DE0CD
:102FA00070E082E992E00E947F17892B11F080E0A7
:102FB00008958091100263E070E081FD03C08FE806
:102FC00092E002C08CE892E00E947F17892B79F78B
:102FD0006DE070E08FE792E00E947F17892B39F750
:102FE0000E947A1FDC01CB01805A9541AF4FBF4F41
:102FF0008093670490936804A0936904B0936A0473
:103000000E94AB1781E0809313028093120210920A
:103010001102089520910F0236E0839FC001112410
:10302000629F800D911D1124811522E0920714F0FA
:1030300080E090E089599D4F90936C0480936B04DD
:10304000089520916B0430916C04215632404091D8
:103050000F02642F70E0C9010E947D26481B463094
:1030600010F4240F311D211582E0380710F020E004
:1030700030E029593D4F30936C0420936B04089540
:10308000CF93DF938A3011F481E003C08D3029F4AF
:1030900080E0DF91CF910C94B618C62F682F8091F5
:1030A0006B0490916C0426E0FC01A9EEB1E0019064
:1030B0000D922A95E1F7603E30F026E0FC01119276
:1030C0002A95E9F70AC0F6E06F9FB0011124615616
:1030D0007D4F46E050E00E949726C11135C0C09157
:1030E0006B04D0916C0446E050E0BE0189EE91E0A3
:1030F0000E94A026892BB1F1C756D2409E0185E0DF
:10310000369527958A95E1F781E090E0AC0102C001
:10311000440F551F2A95E2F72091140230911502B1
:10312000242B352B259645E0D695C7954A95E1F792
:1031300002C0880F991FCA95E2F7822B932B9093B8
:103140001502809314020EC0E0916B04F0916C04A0
:103150009F012A5F3F4F2E173F0709F2808180951C
:103160008193F9CFDF91CF910C942118CF93E82F61
:1031700020916B0430916C042756324040910F022D
:10318000642F70E0C9010E947D26481B842FEE2326
:1031900059F066E00E947126C82FC150B0F060E07F
:1031A00080E20E944018F9CFA901480F511D411536
:1031B000524018F080E020E030E0280F311D2959FE
:1031C0003D4F30936C0420936B04CF9108951F936F
:1031D000CF93DF93EC01162FFE018491882329F011
:1031E000612F0E9440182196F7CFDF91CF911F9158
:1031F00008950E94E71881E00C94B618809113029C
:103200008823F9F00E947A1FDC01CB01805A954196
:10321000AF4FBF4F8093670490936804A0936904F5
:10322000B0936A048091120281110BC062E070E0D9
:103230008DE792E00E947F17892B19F481E080933B
:1032400012028091120208956F927F928F929F9244
:10325000AF92BF92CF92DF92EF92FF920F931F93A4
:10326000CF93DF9380911302882309F4DCC020916F
:103270001402309115022115310509F4D4C0809152
:1032800011028111D0C061E070E0082F10E03B0115
:10329000082E02C0660C771C0A94E2F7A9014621A9
:1032A0005721452B11F48F5FF0CF909110029801B8
:1032B00065E0220F331F6A95E1F790FD12C08295F9
:1032C000880F807680930B01220F232F221F330B50
:1032D000319520930E01815E80930C0110920F01B5
:1032E00012C045E0369527954A95E1F7220F220F47
:1032F000220F20930B0110920E01295F20930C01E5
:1033000083E080930F0124E630E047E050E069E07D
:1033100071E088E70E94611D892B09F084C08091CB
:10332000100280FD23C0A80195E0440F551F9A9517
:10333000E1F749595D4F04E610E020E230E060E437
:1033400088E70E94881D892B09F06DC00E94FE1835
:10335000E301C095D0958091140290911502C82385
:10336000D923D0931502C09314025DC080E2EFEE22
:10337000F1E0DF011D928A95E9F785E0000F111F4A
:103380008A95E1F7AFE2B1E04BE251E099249394E2
:103390002D91EA018991AE01B801680F711D69593B
:1033A0007D4F30E021513E4FF90197E07F01E21A55
:1033B000F30AA92C01C0AA0CEA94EAF77B01B12C0C
:1033C000E70189917E018A21892E8B18D82DD7702B
:1033D000CD2E0D2E000CDD08C82F01C0CC0FDA95C4
:1033E000EAF7D194C194D108D7E0CD22DD2401C001
:1033F0008695CA94EAF78C2BD0808D298083B3946C
:1034000088E0B812DDCF915031969F3F79F6C1E048
:10341000A333BC0709F0BCCF04E610E020E230E0A3
:103420004FEE51E08CCFDF91CF911F910F91FF9024
:10343000EF90DF90CF90BF90AF909F908F907F9054
:103440006F9008958091130290911202882389F061
:10345000992369F062E070E08BE792E00E947F17A9
:10346000892B19F080911202089510921202909106
:10347000120281E0892708950C94B5040F931F93DD
:1034800080911302882329F160E080E00E940A18ED
:103490000E943C1A0E942419809112028823C9F0CC
:1034A0000E947A1F009167041091680420916904BA
:1034B00030916A04DC01CB01801B910BA20BB30B92
:1034C0008F3F9F4FAF4FBF4720F41F910F910C9438
:1034D000221A1F910F910895CF93DF93EC01FB0106
:1034E0008281882309F43CC1C430FDE5DF0760F424
:1034F000CB3F9CE5D90788F49E0122503C452431FE
:10350000310508F02EC109C0C236EDE5DE0729F00D
:10351000C63AFDE5DF0709F024C10E94880F9093A9
:10352000450280934402C1318CE5D80709F4C6C036
:1035300008F042C0C930ECE5DE0709F49BC000F595
:10354000C5308CE5D80709F485C078F4C330ECE5C4
:10355000DE0709F478C008F07AC0C230DC4509F013
:10356000F5C0809144028160EFC0C7309CE5D90767
:1035700009F478C008F07AC0809144028061E4C008
:10358000CD30FCE5DF0709F487C058F4CB309CE56B
:10359000D90709F479C008F07BC0809144028860A3
:1035A0006FC0CF30FCE5DF0709F480C008F082C0AF
:1035B00080914402877FC8C0CE3F9CE5D90709F4BB
:1035C00071C000F5C531FCE5DF0709F485C068F47A
:1035D000C3319CE5D90709F475C008F095C00E9475
:1035E0003F09809144028F77AFC0CC3FFCE5DF07F5
:1035F000A9F108F054C0CB3FDC4509F0A7C0809189
:10360000450240C0C230EDE5DE0709F489C058F438
:10361000C1158DE5D80709F45AC008F069C080913A
:10362000450282602FC0C236EDE5DE0709F47CC09A
:10363000C63AFDE5DF0709F481C0C330DD4509F076
:1036400085C080E06EC08091440282607DC0809120
:10365000440216C080914402886076C08091450281
:1036600082604FC08091440280626EC080914402AB
:1036700080646AC00E943F0980914402806864C0EF
:10368000846062C081603DC0809144028E7F5CC0D6
:10369000809144028D7F58C08091440216C0809171
:1036A000450218C0809145028D7F2BC08091440255
:1036B0008F7E4AC0809144028F7D46C08091440233
:1036C0008F7B42C080914402877F8B7F3DC0809179
:1036D00045028D7F8E7F15C08091440282FB222798
:1036E00020F991E0922790FB82F990FB83F92CC09E
:1036F00080914502982F909591708E7F892B90FB39
:1037000081F98093450222C00E943F0980914402C2
:1037100087FB222720F991E0922790FB87F914C0BC
:1037200081E00E941F1012C08091440284FB222776
:1037300020F991E0922790FB84F906C08091440221
:10374000982F909590FB80F98093440280914402D9
:10375000909145020E94990F0E943F0980E001C0AC
:1037600081E0DF91CF910895CF93DF9386319C451F
:1037700041F5EB010E94920E982F8A81209102015F
:1037800030910301882379F09A7A81E009F480E08E
:1037900080931602911102C069E201C065E3C9017C
:1037A0000E94AB1E0AC080911602811102C069E21C
:1037B00001C065E3C9010E94B61E0E94D40E80E0DC
:1037C00001C081E0DF91CF9108950F931F93CF93B4
:1037D000DF93C42FD22FFC0182818823C9F040934C
:1037E00019020E946E1F909318028093170280E2C4
:1037F0008C0F883008F057C0C77081E001C0880F77
:10380000CA95EAF7DF91CF911F910F910C94D106E1
:1038100080911902481330C08091170290911802CC
:103820000E94861F883C910538F510E21D0FCD17C8
:10383000B9F080E28C0F883040F4C77081E001C09D
:10384000880FCA95EAF70E94D806183028F581E05B
:103850009D2F977001C0880F9A95EAF70E94D106B4
:10386000802F0E94C8061830F0F4D77081E001C0A4
:10387000880FDA95EAF70AC080E28C0F883098F456
:10388000C77081E001C0880FCA95EAF7DF91CF9138
:103890001F910F910C94D806802FDF91CF911F912B
:1038A0000F910C94C806DF91CF911F910F9108954D
:1038B0000F939C01CB01243F4CE5340731F188F490
:1038C000293DFCE53F07D9F02A3D4CE5340779F165
:1038D000283D3C45A9F506E221EE41EE68ED7CE588
:1038E0002BC0263FFCE53F07E1F0A8F0273F3C4511
:1038F00039F507E225EE46EE67EF7CE51DC007E2ED
:1039000025EE45EE69ED7CE517C006E221EE40EEBE
:1039100064EF7CE511C007E225EE44EE65EF7CE53F
:103920000BC006E221EE42EE66EF7CE505C008E240
:1039300021E045EE6AED7CE50E94E51B80E008C0D1
:10394000FC018281882319F01092190201C081E0E4
:103950000F9108951092B9008CE08093B8000895FB
:103960009F92AF92BF92CF92DF92EF92FF920F930E
:103970001F93CF93DF93B82EEB010E946E1F6C0153
:10398000C431D10558F0CF3F8FEFD80759F0CE01A1
:1039900064E170E00E947D267B0107C0EE24E39481
:1039A000F12C03C025E0E22EF12C84E8A82E94EA45
:1039B000992E1092BC009092BC000E946E1F8C0148
:1039C0008091BC0087FD08C00E946E1F801B910B78
:1039D0008E159F05A8F32AC08091B900887F883092
:1039E00041F08091B900887F803119F00FEF1FEF0F
:1039F0001FC0B092BB00A092BC000E946E1F8C0141
:103A00008091BC0087FD08C00E946E1F801B910B37
:103A10008E159F05A8F30AC08091B900887F883170
:103A200011F0803419F700E010E00EC00EEF1FEF28
:103A3000CF3F8FEFD80709F4BCCFC6010E94861F85
:103A40008C179D0708F4B5CFC801DF91CF911F9166
:103A50000F91FF90EF90DF90CF90BF90AF909F902D
:103A600008950F931F93CF93DF93EB018093BB00D7
:103A700084E88093BC000E946E1F8C018091BC0082
:103A800087FD0EC0CF3F8FEFD807C1F30E946E1F96
:103A9000801B910B8C179D0788F38EEF9FEF0CC056
:103AA0002091B900287F81E090E0283211F480E075
:103AB00090E0919581959109DF91CF911F910F91A0
:103AC0000895CF92DF92EF92FF920F931F93CF93BF
:103AD000DF936B018A017901B9010E94B01CE601F4
:103AE0000C0D1D1DC017D10761F424E92093BC0003
:103AF000DF91CF911F910F91FF90EF90DF90CF90CA
:103B0000089597FDF2CFB70189910E94311DEACF48
:103B1000CF92DF92EF92FF920F931F93CF93DF9399
:103B2000C62F6A017901B8010E94B01C97FD11C02F
:103B3000B8018C2F0E94311DE601EC0CFD1CCE1546
:103B4000DF0539F097FD05C0B80189910E94311D4C
:103B5000F6CF24E92093BC00DF91CF911F910F9104
:103B6000FF90EF90DF90CF90089584E98093BC00A0
:103B700008959093350180933401089590931F0226
:103B800080931E020895E0911E02F0911F0230976B
:103B900021F00190F081E02D099480E00895E091FA
:103BA0001E02F0911F02309799F020911C012223F0
:103BB00059F02091440227FF07C0DC012C91119697
:103BC0002C93119726E02C930280F381E02D099429
:103BD000089520911C0230911D022817390771F0B9
:103BE00090931D0280931C02E0911E02F0911F022F
:103BF000309721F00680F781E02D099408952091F7
:103C00001A0230911B022817390771F090931B029A
:103C100080931A02E0911E02F0911F02309721F06A
:103C20000084F185E02D09940895FC01329680917D
:103C30001C01882331F08091440287FF02C09EE17D
:103C400001C096E080E0915028F021912223D9F321
:103C50008F5FF9CF0895662351F120911C01222333
:103C6000E9F02091440227FF19C0462F469546955A
:103C700046954E31E0F4677021E030E002C0220F3B
:103C8000331F6A95E2F7FC01E40FF11D828190E099
:103C90002823392381E0232B69F409C0FC013296E3
:103CA00008962191621729F0E817F907D1F780E00B
:103CB000089581E008959C01FC0132969FEF80E019
:103CC0004191461789F09F3F19F4411101C0982F87
:103CD0008F5F8630A9F79F3F39F0F901E90FF11D99
:103CE00097FDFA956283089508959C012A5F3F4FDE
:103CF000FC014281461301C012820196821793078C
:103D0000B9F70895262F2695269526952E3168F425
:103D1000FC01E20FF11D677021E030E001C0220FCD
:103D20006A95EAF78281282B22830895262F26950B
:103D3000269526952E3170F4FC01E20FF11D677077
:103D400021E030E001C0220F6A95EAF720958281D8
:103D500028232283089520911C01222329F02091F9
:103D6000440227FD0C94821E0C945B1E20911C01C2
:103D7000222329F02091440227FD0C94961E0C94D6
:103D8000751E20911C01FC013296222331F0809196
:103D9000440287FF02C08EE101C086E0DF011D9270
:103DA0008A95E9F7089508950C94D31E83E08093D3
:103DB00020020C94D41E811102C081E001C082E077
:103DC000809320020C94D41E0C94DB1E81E080931F
:103DD00020020C94D41E0C94E61E08950C94ED1E43
:103DE0000C94EE1E0C94ED1E0C94ED1E0C94ED1E26
:103DF000CF930E94F41E0E94D1130E94F21EC0E0D5
:103E00008C2F0E940913811104C0CF5FC530C1F708
:103E100001C081E0CF91089508951F920F920FB6CF
:103E20000F9211248F939F93AF93BF9380912102A0
:103E3000811113C080916D0490916E04A0916F0464
:103E4000B09170044196A11DB11D80936D049093B3
:103E50006E04A0936F04B0937004BF91AF919F91D3
:103E60008F910F900FBE0F901F9018958091750441
:103E7000843031F10E9485051092210220E488E10E
:103E800090E00FB6F894A895809360000FBE209341
:103E9000600083B7817F846083BF83B7816083BF05
:103EA0007894889583B78E7F83BF0FB6F894A895D2
:103EB00080916000886180936000109260000FBE66
:103EC00008950E943F090C948B0582E084BD93E025
:103ED00095BD9AEF97BD80936E0008952FB7F89423
:103EE00080916D0490916E04A0916F04B091700464
:103EF0002FBF08952FB7F89460916D0470916E04F0
:103F000080916F04909170042FBF08959C014FB76A
:103F1000F89480916D0490916E04A0916F04B0911B
:103F200070044FBF821B930B089578941F920F92D9
:103F30000FB60F9211248F939F93AF93BF938091ED
:103F40006D0490916E04A0916F04B091700401967D
:103F5000A11DB11D80936D0490936E04A0936F0416
:103F6000B0937004BF91AF919F918F910F900FBE4E
:103F70000F901F90189581E08093E00080E280937D
:103F8000D8001092C9008FE19EE40197F1F700C0BC
:103F9000000087E090EBDC0180937E0490937F0427
:103FA000A0938004B09381049CE088E10FB6F8945C
:103FB000A895809360000FBE90936000FFCF809122
:103FC0004202089508950895CF93DF9320911C0134
:103FD000222339F02091440227FF03C060E222E04F
:103FE00002C068E021E02093E9002FEF3091E80063
:103FF000215035FD06C035ED3A95F1F7000021114D
:10400000F5CF2091E80025FF1DC0EC0180911C0137
:10401000811105C040E050E068E070E003C070E04E
:1040200040E050E0CE010E94D3218091E8008E77DD
:104030008093E80080E2FE01A2E2B2E001900D92DE
:104040008A95E1F7DF91CF910895089508958091C1
:104050007404811109C00E9464230E94C1238091CD
:10406000E20084608093E200089510927404089541
:104070000C94EB1E6091710481E0611101C080E03D
:104080000C94D61E9091750481E0943009F080E084
:10409000609171040C94DB1E42E061EC81E00E94AF
:1040A000DD2242E261EC82E00E94DD229091750403
:1040B00081E0943009F080E0609171040C94E41E7A
:1040C00080917704833009F461C030F4813071F05D
:1040D000823009F49AC008958A3009F486C08B3082
:1040E00009F46CC0893009F0A8C020C08091760422
:1040F000813A09F0A2C08091E800877F8093E800B0
:1041000080917A0490917B04892B21F460E282E211
:1041100092E003C060E080E090E070E00E941E2228
:104120008091E8008B778093E80008958091760471
:10413000813209F082C080917A0490917B040297C9
:1041400008F07BC08091E800877F8093E800809131
:10415000E80082FD05C0809175048111F8CF6DC023
:104160002091F3008091F20090E0922B029731F4BD
:104170008091F100813011F0863021F48091F100BE
:10418000809342028091E8008B7753C0809176043F
:10419000813A09F052C080917A0490917B04892B76
:1041A00009F04BC08091E800877F8093E800809100
:1041B000E80080FFFCCF80911C0136C0809176041E
:1041C0008132D9F580917A0490917B04892BA9F5ED
:1041D0008091E800877F8093E8000E9412238091FD
:1041E000780480931C010C943F09809176048132FD
:1041F00021F58091E800877F8093E8000E941223D8
:104200008091790480934302089580917604813AE5
:10421000A1F48091E800877F8093E8008091E80016
:1042200080FFFCCF809143028093F1008091E800F1
:104230008E778093E8000C941223089584B7877FCB
:1042400084BF0FB6F894A895809160008861809330
:104250006000109260000FBE90E080E80FB6F89406
:1042600080936100909361000FBE0C94E61E0E9443
:1042700064230E94C123E2EEF0E0808184608083A9
:1042800078940C94562680E191E00C94BE1D8091A8
:1042900075048530A9F480917504853079F40E9405
:1042A000361F809173048823B1F30E94F81E88237F
:1042B00091F30E94BD210E943F09EDCF0C94611F34
:1042C000089508950C946421292F33272330310554
:1042D000C9F060F42130310581F02230310509F058
:1042E00044C08BE390E023E138E043C02132310544
:1042F000E1F02232310549F138C082E190E02EE44C
:1043000038E037C099278130910549F028F00297AD
:1043100061F5EFEDF7E005C0EFE0F8E002C0EDEF8A
:10432000F7E0849190E09F0124C06115710541F090
:1043300061307105D1F489E090E02EE338E019C0D6
:1043400089E090E025E238E014C06115710541F084
:104350006130710551F48BE390E020E638E009C04C
:1043600080E490E02BE938E004C080E090E020E0B9
:1043700030E0FA0131832083089580E189BD82E134
:1043800089BD09B400FEFDCF8091D8008F7D809358
:10439000D8008091E00082608093E0008091E0008E
:1043A00081FDFCCF0895CF92DF92EF92FF920F93A1
:1043B0001F93CF93DF93EC018B017A010E9431238D
:1043C000811133C0E114F10439F0F701808191814A
:1043D000081B190BC80FD91FC12CD12C01151105B1
:1043E00019F18091E80085FD16C08091E8008E7774
:1043F0008093E800E114F10449F0F7018081918194
:10440000C80ED91ED182C08285E00FC00E94312320
:10441000882321F30AC089918093F100015011098A
:10442000FFEFCF1ADF0ADACF80E0DF91CF911F9143
:104430000F91FF90EF90DF90CF90089520917C0432
:1044400030917D042617370748F06115710539F45E
:104450002091E8002E772093E80001C0B901FC010B
:1044600020E06115710579F1809175048823F1F1DF
:104470008530F1F18091E80083FD3CC08091E80037
:1044800082FD2EC08091E80080FFEBCF2091F300E9
:104490008091F20090E0922B6115710551F0883007
:1044A000910538F421912093F10061507109019632
:1044B000F3CF21E0089709F020E08091E8008E77A3
:1044C0008093E800CECF2111CFCF0AC08091750430
:1044D000882361F0853061F08091E80083FD0AC097
:1044E0008091E80082FFF2CF80E0089582E0089595
:1044F00083E0089581E0089520917C0430917D044B
:104500002617370748F06115710539F42091E80046
:104510002E772093E80001C0B901FC0120E061156D
:10452000710591F180917504882309F440C08530AC
:1045300009F43FC08091E80083FD3DC08091E80010
:1045400082FD2FC08091E80080FFE9CF2091F30029
:104550008091F20090E0922B6115710559F088303E
:10456000910540F424912093F10031966150710936
:104570000196F2CF21E0089709F020E08091E80051
:104580008E778093E800CBCF2111CCCF0AC08091E9
:104590007504882361F0853061F08091E80083FD27
:1045A0000AC08091E80082FFF2CF80E0089582E0A7
:1045B000089583E0089581E00895982F973068F575
:1045C0009093E900981739F07091EC002091ED007C
:1045D0005091F00003C0242F762F50E021FD02C03F
:1045E0009F5FECCF3091EB003E7F3093EB0030913A
:1045F000ED003D7F3093ED003091EB003160309362
:10460000EB007093EC002093ED005093F0002091AC
:10461000EE0027FDE5CF80E008958F708093E900DC
:1046200081E008958091760487FF11C08091E800B1
:1046300082FD05C0809175048111F8CF11C0809171
:10464000E8008B770BC080917504882349F0809136
:10465000E80080FFF8CF8091E8008E778093E80033
:1046600008952091E4003091E50095E64091EC003A
:10467000842F817040FF23C08091E80080FD1DC021
:1046800080917504882399F0853099F08091EB0032
:1046900085FD11C04091E4005091E50024173507D5
:1046A00029F3915011F09A01E1CF84E0089582E05E
:1046B000089583E0089581E0089580E00895409191
:1046C000E80042FFDDCF08950E94D2230E94DA2342
:1046D000E0EEF0E0808181608083E8EDF0E08081B1
:1046E0008F77808319BCA7EDB0E08C918E7F8C937F
:1046F00080818F7E80831092740408950F931F939E
:10470000CF93DF930E94D2230E94DA23C8EDD0E03A
:1047100088818F77888388818068888388818F7D6E
:10472000888319BC1092750410927104109273045E
:104730001092720400EE10E0F80180818B7F80837C
:1047400088818160888342E060E080E00E94DD2211
:10475000E1EEF0E080818E7F8083E2EEF0E0808108
:1047600081608083808188608083F80180818E7F72
:104770008083888180618883DF91CF911F910F9121
:104780000895E8EDF0E080818F7E8083E7EDF0E032
:1047900080818160808384E082BF81E080937404A3
:1047A0000C947E23E8EDF0E080818E7F8083109270
:1047B000E20008951092DA001092E10008951F922D
:1047C0000F920FB60F9211242F933F934F935F9345
:1047D0006F937F938F939F93AF93BF93EF93FF93C9
:1047E0008091E10082FF0BC08091E20082FF07C050
:1047F0008091E1008B7F8093E1000E94552680919B
:10480000DA0080FF1FC08091D80080FF1BC080911C
:10481000DA008E7F8093DA008091D90080FF0DC08E
:1048200080E189BD82E189BD09B400FEFDCF81E050
:10483000809375040E94272005C019BC109275044E
:104840000E9435208091E10080FF19C08091E20034
:1048500080FF15C08091E2008E7F8093E2008091FE
:10486000E20080618093E2008091D80080628093B2
:10487000D80019BC85E0809375040E943A2080918D
:10488000E10084FF30C08091E20084FF2CC080E111
:1048900089BD82E189BD09B400FEFDCF8091D800B9
:1048A0008F7D8093D8008091E1008F7E8093E1001E
:1048B0008091E2008F7E8093E2008091E20081602F
:1048C0008093E20080917104882311F084E007C096
:1048D0008091E30087FD02C081E001C083E0809306
:1048E00075040E9442208091E10083FF29C08091DD
:1048F000E20083FF25C08091E100877F8093E10083
:1049000082E080937504109271048091E1008E7FA3
:104910008093E1008091E2008E7F8093E20080919D
:10492000E20080618093E20042E060E080E00E946B
:10493000DD228091F00088608093F0000E94382092
:10494000FF91EF91BF91AF919F918F917F916F9167
:104950005F914F913F912F910F900FBE0F901F903D
:1049600018951F920F920FB60F9211242F933F9319
:104970004F935F936F937F938F939F93AF93BF9367
:10498000CF93DF93EF93FF93C091E900CF708091B5
:10499000EC00D82FD17080FDD0E81092E900809112
:1049A000F000877F8093F00078940E94F5241092A5
:1049B000E9008091F00088608093F000CD2BCF70EB
:1049C000C093E900FF91EF91DF91CF91BF91AF913B
:1049D0009F918F917F916F915F914F913F912F9117
:1049E0000F900FBE0F901F9018951F93CF93DF93DA
:1049F000CDB7DEB7AA970FB6F894DEBF0FBECDBF16
:104A0000E6E7F4E08091F100819324E0EE37F207CD
:104A1000C9F70E9460208091E80083FF2EC1809139
:104A2000760490917704492F50E04A30510508F000
:104A300024C1FA01EE59FF4F0C949126803821F0E1
:104A4000823809F01AC108C08091720490917304F1
:104A5000992389F082600FC080917A048F7087302B
:104A600008F00BC18093E9008091EB0085FB88275B
:104A700080F91092E9009091E800977F9093E80008
:104A80008093F1001092F100D1C0282F2D7F09F002
:104A9000F4C0882319F0823061F0EFC0809178046F
:104AA000813009F0EAC0933009F080E0809373040C
:104AB0002EC08091780481112AC080917A048F7071
:104AC0002FEF280F263008F0D8C08093E9002091FE
:104AD000EB0020FF1CC0933021F48091EB0080623A
:104AE00014C09091EB0090619093EB0021E030E0D6
:104AF000A90102C0440F551F8A95E2F74093EA00CE
:104B00001092EA008091EB0088608093EB00109295
:104B1000E9008091E800877F8093E8000E941223DB
:104B2000ACC08111AAC0109178041F778091E30076
:104B30008078812B8093E3008091E800877F8093C9
:104B4000E8000E9412238091E80080FFFCCF809152
:104B5000E30080688093E300111102C082E001C08D
:104B600083E08093750489C08058823008F085C046
:104B700080917804909179048C3D53E0950779F504
:104B800083E08A838AE289834FB7F894DE01139623
:104B900020E03EE051E2E32FF0E050935700E49133
:104BA00020FF03C0E295EF703F5FEF708E2F90E023
:104BB000EA3010F0C79601C0C0968D939D932F5F89
:104BC000243149F74FBF8091E800877F8093E80048
:104BD0006AE270E0CE0101960E941E2216C060912A
:104BE0007A0470917B04AE014F5F5F4F0E94622197
:104BF000BC01892B09F441C09091E800977F909304
:104C0000E80089819A810E947C228091E8008B775C
:104C10008093E80032C0803881F58091E800877F7A
:104C20008093E800809171048093F1008091E80006
:104C30008E7772CF811121C0809178049091790490
:104C400099270297D4F48091E800877F8093E80049
:104C500080917804809371040E94122380917104E2
:104C6000811106C08091E30087FD02C081E001C090
:104C700084E0809375040E944C208091E80083FFBB
:104C80000AC08091E800877F8093E8008091EB0064
:104C900080628093EB00AA960FB6F894DEBF0FBE39
:104CA000CDBFDF91CF911F9108950895CF9380914B
:104CB00075048823A1F0C091E900CF709091EC00B9
:104CC000892F817090FD80E8C82B1092E9008091B7
:104CD000E80083FD0E94F524CF70C093E900CF91D6
:104CE0000895991B79E004C0991F961708F0961B48
:104CF000881F7A95C9F780950895AA1BBB1B51E1BF
:104D000007C0AA1FBB1FA617B70710F0A61BB70B3B
:104D1000881F991F5A95A9F780959095BC01CD01E0
:104D20000895EE0FFF1F0590F491E02D0994FB010B
:104D3000DC0102C005900D9241505040D8F7089513
:104D4000FB01DC0104C08D910190801921F44150D8
:104D50005040C8F7881B990B0895F999FECF92BD72
:104D600081BDF89A992780B50895A6E1B0E044E0A6
:104D700050E00C94E726A8E1B0E042E050E00C944B
:104D8000E726262FF999FECF92BD81BDF89A0197AB
:104D900000B4021639F01FBA20BD0FB6F894FA9A83
:104DA000F99A0FBE08950396272F0E94C2260E94EB
:104DB000C126252F0E94C226242F0C94C2260196BC
:104DC000272F0E94C2260C94C126DC01CB01FC01D6
:104DD000F999FECF06C0F2BDE1BDF89A319600B454
:0E4DE0000D9241505040B8F70895F894FFCF5F
:104DEE00C800B30100060006060021007F22000362
:104DFE00DF1FE41F25202620E21FE31F01969734B4
:104E0E003536F695F5F4F1F09400010008101818F7
:044E1E001008000078
:00000001FF
